:100000002E288207003400340034003400341B34BE
:1000100077344034003435346734E03400346A34A3
:10002000CF34C03400349A341D3420340034D534F5
:100030009F34803401341334B234203401344034DA
:100040006F34403401347B34CA3490340134AB34DF
:100050003F3400340134C934C33480348B018316F7
:100060008117FF30850086018312A5208519392864
:100070003F21890199220808A30099220808A400B9
:1000800099220808A50099220808A60028308C00AB
:1000900001308D00D6308E0000308F00F3212122F8
:1000A000A321D9210508B30003303305B200B00104
:1000B0004030AF00B401B7011521B31D7B289D016D
:1000C0009C019B0101309A0033197028E8309A0096
:1000D00003309B00702803109A0D9B0D9C0D9D0D05
:1000E000AF0DB00D031C6B28B418782802218E28A0
:1000F000C520DD208E28B41887280430B702D730F9
:100100003707031C85282830B70093208E28043039
:10011000B707D73037070318B7019320F3212122FF
:10012000A321D9215C28370801208F00B70A37089E
:1001300001208E00B70A370801208D00B70A370862
:1001400001208C000330B7020800A1223030860065
:100150008615A1228611303086008615A4228611CC
:10016000303086008615A422861120308600861540
:10017000A722861128306A2208306A2201306A22BA
:1001800006306A220C306A2208001A088C07031C09
:10019000CE288D0FCE288E0FCE288F0A1B088D07F4
:1001A000031CD5288E0FD5288F0A1C088E07031C28
:1001B000DA288F0A1D088F070800FE300F07031882
:1001C000F92801300F02031C012936300E070318ED
:1001D000F928C9300E02031C01293C300D07031811
:1001E000F928C3300D02031C012980300C02031CC6
:1001F000012980308C00C3308D00C9308E00013061
:100200008F0008009A099B099C099D099A0F0D29E6
:100210009B0F0D299C0F0D299D0AC5208F1F1429A6
:100220008C018D018E018F010800B0014030AF00BC
:100230006400B01B1F290830AF070318B00A050877
:10024000B30003303305B100320603191829031037
:10025000B20D3108B20632080239B500340603196E
:1002600036293508B4003108B2001829B2183A29E5
:10027000B4013C290230B4003108B20008008030DB
:100280008C0096308D0098308E0000308F008901F0
:1002900099220808A30099220808A40099220808B6
:1002A000A50099220808A600F3212122C430AB0042
:1002B0006A224330AB006E224130AB006E224C30DC
:1002C000AB006E22A321D92115219D019C019B0128
:1002D00010309A0033196E2980309A000000B4184B
:1002E0007C299A099B099C099D099A0F7C299B0FDF
:1002F0007C299C0F7C299D0A1A08A307031C8529C9
:10030000A40F8529A50F8529A60A1B08A407031C8D
:100310008C29A50F8C29A60A1C08A507031C912966
:10032000A60A1D08A607B31D6229890123088800B3
:100330008C22240888008C22250888008C2226081C
:1003400088008C2208009501960197019801990177
:100350002030A0002308A7002408A8002508A90031
:100360002608AA000310271CCC290C089607031C9A
:10037000BE29970FBE29980FBE29990A0D08970725
:10038000031CC529980FC529990A0E089807031C54
:10039000CA29990A0F089907990C980C970C960C82
:1003A000950CAA0CA90CA80CA70CA00BB2299901BA
:1003B0000800153084000008A2000830A100A20C3B
:1003C000031CE629861786168612E92986138616E7
:1003D0008612A10BDF29840A1A300402031CDB29D0
:1003E00006140610080020309E0090019101920131
:1003F0009301940103108C0D8D0D8E0D8F0D03183C
:100400000C14900D910D920D930D940D9E03031DF0
:100410000A2A0800103084001622840A1622840A50
:100420001622840A1622840A1622FA2903300007AB
:100430009F009F198000303000079F009F1B8000A5
:10044000080081306A22130E0F39303E6E221308E5
:100450000F39303E6E222C306E22120E0F39303E94
:100460006E2212080F39303E6E22110E0F39303EC7
:100470006E222E306E22C0306A2211080F39303EB3
:100480006E22100E0F39303E6E2210080F39303EAA
:100490006E2220306E226B306E2248306E227A300F
:1004A0006E22080086018316F030860083128610C3
:1004B0000615FF30AD0086150608AC008611000059
:1004C0000000861500008611AD030319692AAC1BD4
:1004D0005B2A0800AB00B8018610712AAB00381403
:1004E000861452228601831600308600831206117C
:1004F0008610381886140F3086052B08F0398604CC
:100500008615000086110F3086052B0EF039860403
:1005100086150000861108008316081555308900DD
:10052000AA30890088148818932A08118312890A2E
:100530000800831608148312890A0800FF30AD00F2
:10054000AC2A8030AD00AC2A4030AD00AC2A20305F
:10055000AD00AC2A1030AD00FF30AE00AE0BAE2ABD
:06056000AD0BAC2A0800FF
:084000007F007F007F007F00BC
:02400E00F53F7C
:10420000C4001D00F3002A000000000000000000B0
:10421000000000000000000000000000000000009E
:10422000000000000000000000000000000000008E
:10423000000000000000000000000000000000007E
:10424000000000000000000000000000000000006E
:10425000000000000000000000000000000000005E
:10426000000000000000000000000000000000004E
:10427000000000000000000000000000000000003E
:00000001FF
